:020000040000FA
:020000002D28A9
:040002000034003492
:08000800B700030EB8000C1054
:1000100005190D28301431100F28311430101C3000
:10002000B522AF002F1D28282F1C1C283008013AAC
:10003000B0003108013AB1000C30B522AC002C1CE4
:100040002828301C26288512051628280512851612
:10005000380E8300B70E370E09008501073099006E
:1000600083169F0170308F000F3085000C148312AF
:10007000113090000B178B178501B401A201A30169
:10008000A401A501A601A701A001A10105195928F4
:1000900005195B2800302002031946281030200281
:1000A00003185F28A10A0C30210203196228A0015D
:1000B00046280000000000000000A00A4628A00119
:1000C000A1014628A001A10105197228051974286B
:1000D0000030200203196428103020020318782809
:1000E000A00164280000000000000000A00A6428AD
:1000F0008E018F01A001A101A115051990280519F4
:1001000092280030200203197D28103020020318A5
:100110009628A20D2214A10B8E289A28A0017D28D2
:100120000000000000000000A00A7D28A20D22109F
:10013000A10B8E28A001A1010519AA280519AC2838
:100140000030200203199C28103020020318B02828
:10015000A0013E280000000000000000A00A9C282A
:10016000A001A101A1150519C6280519C82800304C
:1001700020020319B328103020020318CC28A30D45
:100180002314A10BC428D028A001B328000000002C
:1001900000000000A00AB328A30D2310A10BC4285F
:1001A000A001A1010519E0280519E228003020026C
:1001B0000319D228103020020318E628A0013E2897
:1001C0000000000000000000A00AD228A001A10148
:1001D000A1150519FC280519FE2800302002031975
:1001E000E9281030200203180229A40D2414A10BC1
:1001F000FA280629A001E9280000000000000000FC
:10020000A00AE928A40D2410A10BFA28A001A1013D
:100210000519162905191829003020020319082983
:100220001030200203181C29A001A829000000009A
:1002300000000000A00A0829A001A101A1150519CC
:100240003229051934290030200203191F291030E2
:10025000200203183829A50D2514A10B30293C29AB
:10026000A0011F290000000000000000A00A1F29B3
:10027000A50D2510A10B3029A001A10105194C29BC
:1002800005194E290030200203193E2910302002A2
:1002900003185229A001A829000000000000000056
:1002A000A00A3E29A001A101A11505196829051977
:1002B0006A29003020020319552910302002031842
:1002C0006E29A60D2614A10B66297229A0015529B5
:1002D0000000000000000000A00A5529A60D26100D
:1002E000A10B6629A001A1010519822905198429FC
:1002F00000302002031974291030200203188829C5
:10030000A001A8290000000000000000A00A742934
:10031000A001A101A11505199E290519A0290030E8
:10032000200203198B29103020020318A429A70DDD
:100330002714A10B9C29A829A0018B2900000000EB
:1003400000000000A00A8B29A70D2710A10B9C29F3
:10035000220823062406250626062706031D3E2816
:100360002209031DB529B4013E28220803199E2A3B
:10037000A21BCA297039703A0319592AB4011C30DA
:10038000B522AF00AF1A3E280030B5222206031D69
:100390003E28E429B4011C30B522AF00AF1E3E2830
:1003A0002208193E03183E281030B5222206031DEC
:1003B0003E281130B5222306031D3E282408A30041
:1003C0002508A4002608A5002308E039B600203A35
:1003D0000319222A3608803A0319362A3608E03AE9
:1003E00003194C2A3608003A03199E2A3608403A67
:1003F0000319032A3608603A0319032A3608A03A7B
:100400000319482A3E281C30B522AF002F1C0B2AA6
:100410002308203AA300AF181A2A231E172AA31E66
:10042000142A85160512192A05168512192A05128D
:1004300085122316A31A1F2A301431103E283114B6
:1004400030103E283F302302031D3E281C30B522C9
:10045000AF002F1C2E2A2408FF3AA400A41B332A25
:10046000301431103E28311430103E281C30B52293
:10047000AF00AF1C3E28231E452A311C422A851698
:1004800005123E28051685123E28051285123E28C3
:10049000A31E4B2A3E283E28EC302302031D3E2893
:1004A000073024060319C02A2508B5002408A52210
:1004B0003C28341CBE29221D6C2AA2183E28221C6E
:1004C000892A622A2308B200B2030310B20D031076
:1004D000B20DB414DB223E28B41C3E282208033996
:1004E0003207B300073033060319BB2AA21D802A46
:1004F0002308B5003308A522B301B401DB223E284E
:100500003308B5222302031D3E28B301B401DB22C8
:100510003E28B41C3E28A21D952A2308B5001C3095
:10052000A522B201B401DB223E281C30B5222302F1
:10053000031D3E28B201B401DB223E282208230617
:10054000031D3E28341485013E2883169B00831228
:10055000350883169A001C1555309D00AA309D0061
:100560009C149C18B12A8312080083169B001C144B
:100570001A088312080008302306031DD82AC42A4B
:1005800008302506031D3E280330B5000030A522A3
:100590000130B5000C30A522C030B5001030A522C6
:1005A0008030B5001130A5220230B5001C30A522E4
:1005B000B20134103C28FF308500EA22EA22EA2208
:1005C000EA22EA22EA22850108000530B900B90BC7
:1005D000E72A08005330BA00E522EE2ABA0BEC2ACB
:1005E000000008003C30BB00EA22BB0BF42A0800E4
:02400E00C43BB1
:104200000300000000000000FF0000001E001D0071
:104210000400000000000000010000000000000099
:10422000C00080000000000000000000000000004E
:10423000000000000000000002000000000000007C
:10424000000000000000000000000000000000006E
:10425000000000000000000000000000000000005E
:04426000000000005A
:00000001FF
